Archive member included because of file (symbol)

c:/freescale/kds_3.0.0/toolchain/bin/../lib/gcc/arm-none-eabi/4.8.4/armv6-m\libgcc.a(_udivsi3.o)
                              ./07_Soft_Component/printf/printf.o (__aeabi_uidiv)
c:/freescale/kds_3.0.0/toolchain/bin/../lib/gcc/arm-none-eabi/4.8.4/armv6-m\libgcc.a(_divsi3.o)
                              ./07_Soft_Component/printf/printf.o (__aeabi_idiv)
c:/freescale/kds_3.0.0/toolchain/bin/../lib/gcc/arm-none-eabi/4.8.4/armv6-m\libgcc.a(_dvmd_tls.o)
                              c:/freescale/kds_3.0.0/toolchain/bin/../lib/gcc/arm-none-eabi/4.8.4/armv6-m\libgcc.a(_udivsi3.o) (__aeabi_idiv0)
c:/freescale/kds_3.0.0/toolchain/bin/../lib/gcc/arm-none-eabi/4.8.4/armv6-m\libgcc.a(_arm_cmpdf2.o)
                              ./07_Soft_Component/printf/printf.o (__aeabi_dcmplt)
c:/freescale/kds_3.0.0/toolchain/bin/../lib/gcc/arm-none-eabi/4.8.4/armv6-m\libgcc.a(_aeabi_uldivmod.o)
                              ./07_Soft_Component/printf/printf.o (__aeabi_uldivmod)
c:/freescale/kds_3.0.0/toolchain/bin/../lib/gcc/arm-none-eabi/4.8.4/armv6-m\libgcc.a(_fixunsdfsi.o)
                              ./07_Soft_Component/printf/printf.o (__aeabi_d2uiz)
c:/freescale/kds_3.0.0/toolchain/bin/../lib/gcc/arm-none-eabi/4.8.4/armv6-m\libgcc.a(_fixunsdfdi.o)
                              ./07_Soft_Component/printf/printf.o (__aeabi_d2ulz)
c:/freescale/kds_3.0.0/toolchain/bin/../lib/gcc/arm-none-eabi/4.8.4/armv6-m\libgcc.a(bpabi.o)
                              c:/freescale/kds_3.0.0/toolchain/bin/../lib/gcc/arm-none-eabi/4.8.4/armv6-m\libgcc.a(_aeabi_uldivmod.o) (__gnu_uldivmod_helper)
c:/freescale/kds_3.0.0/toolchain/bin/../lib/gcc/arm-none-eabi/4.8.4/armv6-m\libgcc.a(eqdf2.o)
                              c:/freescale/kds_3.0.0/toolchain/bin/../lib/gcc/arm-none-eabi/4.8.4/armv6-m\libgcc.a(_arm_cmpdf2.o) (__eqdf2)
c:/freescale/kds_3.0.0/toolchain/bin/../lib/gcc/arm-none-eabi/4.8.4/armv6-m\libgcc.a(gedf2.o)
                              c:/freescale/kds_3.0.0/toolchain/bin/../lib/gcc/arm-none-eabi/4.8.4/armv6-m\libgcc.a(_arm_cmpdf2.o) (__gedf2)
c:/freescale/kds_3.0.0/toolchain/bin/../lib/gcc/arm-none-eabi/4.8.4/armv6-m\libgcc.a(ledf2.o)
                              c:/freescale/kds_3.0.0/toolchain/bin/../lib/gcc/arm-none-eabi/4.8.4/armv6-m\libgcc.a(_arm_cmpdf2.o) (__ledf2)
c:/freescale/kds_3.0.0/toolchain/bin/../lib/gcc/arm-none-eabi/4.8.4/armv6-m\libgcc.a(muldf3.o)
                              ./07_Soft_Component/printf/printf.o (__aeabi_dmul)
c:/freescale/kds_3.0.0/toolchain/bin/../lib/gcc/arm-none-eabi/4.8.4/armv6-m\libgcc.a(subdf3.o)
                              ./07_Soft_Component/printf/printf.o (__aeabi_dsub)
c:/freescale/kds_3.0.0/toolchain/bin/../lib/gcc/arm-none-eabi/4.8.4/armv6-m\libgcc.a(fixdfsi.o)
                              c:/freescale/kds_3.0.0/toolchain/bin/../lib/gcc/arm-none-eabi/4.8.4/armv6-m\libgcc.a(_fixunsdfsi.o) (__aeabi_d2iz)
c:/freescale/kds_3.0.0/toolchain/bin/../lib/gcc/arm-none-eabi/4.8.4/armv6-m\libgcc.a(floatunsidf.o)
                              ./07_Soft_Component/printf/printf.o (__aeabi_ui2d)
c:/freescale/kds_3.0.0/toolchain/bin/../lib/gcc/arm-none-eabi/4.8.4/armv6-m\libgcc.a(_clzsi2.o)
                              c:/freescale/kds_3.0.0/toolchain/bin/../lib/gcc/arm-none-eabi/4.8.4/armv6-m\libgcc.a(muldf3.o) (__clzsi2)
c:/freescale/kds_3.0.0/toolchain/bin/../lib/gcc/arm-none-eabi/4.8.4/armv6-m\libgcc.a(_muldi3.o)
                              c:/freescale/kds_3.0.0/toolchain/bin/../lib/gcc/arm-none-eabi/4.8.4/armv6-m\libgcc.a(bpabi.o) (__aeabi_lmul)
c:/freescale/kds_3.0.0/toolchain/bin/../lib/gcc/arm-none-eabi/4.8.4/armv6-m\libgcc.a(_divdi3.o)
                              c:/freescale/kds_3.0.0/toolchain/bin/../lib/gcc/arm-none-eabi/4.8.4/armv6-m\libgcc.a(bpabi.o) (__divdi3)
c:/freescale/kds_3.0.0/toolchain/bin/../lib/gcc/arm-none-eabi/4.8.4/armv6-m\libgcc.a(_udivdi3.o)
                              c:/freescale/kds_3.0.0/toolchain/bin/../lib/gcc/arm-none-eabi/4.8.4/armv6-m\libgcc.a(bpabi.o) (__udivdi3)
c:/freescale/kds_3.0.0/toolchain/bin/../lib/gcc/arm-none-eabi/4.8.4/../../../../arm-none-eabi/lib/armv6-m\libg.a(lib_a-memset.o)
                              ./07_Soft_Component/printf/printf.o (memset)
c:/freescale/kds_3.0.0/toolchain/bin/../lib/gcc/arm-none-eabi/4.8.4/../../../../arm-none-eabi/lib/armv6-m\libg.a(lib_a-strlen.o)
                              ./07_Soft_Component/printf/printf.o (strlen)

Allocating common symbols
Common symbol       size              file

AlarmTimes          0x4               ./08_Source/isr.o
SecondTimes         0x4               ./08_Source/isr.o
g_time              0x3               ./08_Source/isr.o

Discarded input sections

 .group         0x00000000        0x8 ./08_Source/isr.o
 .group         0x00000000        0x8 ./08_Source/isr.o
 .group         0x00000000        0x8 ./08_Source/isr.o
 .group         0x00000000        0x8 ./08_Source/isr.o
 .group         0x00000000        0x8 ./08_Source/isr.o
 .group         0x00000000        0x8 ./08_Source/isr.o
 .group         0x00000000        0x8 ./08_Source/isr.o
 .group         0x00000000        0x8 ./08_Source/isr.o
 .group         0x00000000        0x8 ./08_Source/isr.o
 .group         0x00000000        0x8 ./08_Source/isr.o
 .group         0x00000000        0x8 ./08_Source/isr.o
 .group         0x00000000        0x8 ./08_Source/isr.o
 .group         0x00000000        0x8 ./08_Source/isr.o
 .group         0x00000000        0x8 ./08_Source/isr.o
 .group         0x00000000        0x8 ./08_Source/isr.o
 .group         0x00000000        0x8 ./08_Source/isr.o
 .group         0x00000000        0x8 ./08_Source/isr.o
 .group         0x00000000        0x8 ./08_Source/isr.o
 .text          0x00000000        0x0 ./08_Source/isr.o
 .data          0x00000000        0x0 ./08_Source/isr.o
 .bss           0x00000000        0x0 ./08_Source/isr.o
 .group         0x00000000        0x8 ./08_Source/main.o
 .group         0x00000000        0x8 ./08_Source/main.o
 .group         0x00000000        0x8 ./08_Source/main.o
 .group         0x00000000        0x8 ./08_Source/main.o
 .group         0x00000000        0x8 ./08_Source/main.o
 .group         0x00000000        0x8 ./08_Source/main.o
 .group         0x00000000        0x8 ./08_Source/main.o
 .group         0x00000000        0x8 ./08_Source/main.o
 .group         0x00000000        0x8 ./08_Source/main.o
 .group         0x00000000        0x8 ./08_Source/main.o
 .group         0x00000000        0x8 ./08_Source/main.o
 .group         0x00000000        0x8 ./08_Source/main.o
 .group         0x00000000        0x8 ./08_Source/main.o
 .group         0x00000000        0x8 ./08_Source/main.o
 .group         0x00000000        0x8 ./08_Source/main.o
 .group         0x00000000        0x8 ./08_Source/main.o
 .group         0x00000000        0x8 ./08_Source/main.o
 .group         0x00000000        0x8 ./08_Source/main.o
 .text          0x00000000        0x0 ./08_Source/main.o
 .data          0x00000000        0x0 ./08_Source/main.o
 .bss           0x00000000        0x0 ./08_Source/main.o
 .debug_macro   0x00000000      0x7f6 ./08_Source/main.o
 .debug_macro   0x00000000       0x16 ./08_Source/main.o
 .debug_macro   0x00000000       0x16 ./08_Source/main.o
 .debug_macro   0x00000000       0x44 ./08_Source/main.o
 .debug_macro   0x00000000      0x209 ./08_Source/main.o
 .debug_macro   0x00000000       0x3a ./08_Source/main.o
 .debug_macro   0x00000000       0x3a ./08_Source/main.o
 .debug_macro   0x00000000       0x26 ./08_Source/main.o
 .debug_macro   0x00000000      0x306 ./08_Source/main.o
 .debug_macro   0x00000000       0x10 ./08_Source/main.o
 .debug_macro   0x00000000     0x839f ./08_Source/main.o
 .debug_macro   0x00000000       0x4c ./08_Source/main.o
 .debug_macro   0x00000000       0x2e ./08_Source/main.o
 .debug_macro   0x00000000       0x9a ./08_Source/main.o
 .debug_macro   0x00000000       0x52 ./08_Source/main.o
 .debug_macro   0x00000000       0x28 ./08_Source/main.o
 .debug_macro   0x00000000       0x22 ./08_Source/main.o
 .debug_macro   0x00000000       0x16 ./08_Source/main.o
 .group         0x00000000        0x8 ./07_Soft_Component/printf/printf.o
 .group         0x00000000        0x8 ./07_Soft_Component/printf/printf.o
 .group         0x00000000        0x8 ./07_Soft_Component/printf/printf.o
 .group         0x00000000        0x8 ./07_Soft_Component/printf/printf.o
 .group         0x00000000        0x8 ./07_Soft_Component/printf/printf.o
 .group         0x00000000        0x8 ./07_Soft_Component/printf/printf.o
 .group         0x00000000        0x8 ./07_Soft_Component/printf/printf.o
 .group         0x00000000        0x8 ./07_Soft_Component/printf/printf.o
 .group         0x00000000        0x8 ./07_Soft_Component/printf/printf.o
 .group         0x00000000        0x8 ./07_Soft_Component/printf/printf.o
 .group         0x00000000        0x8 ./07_Soft_Component/printf/printf.o
 .group         0x00000000        0x8 ./07_Soft_Component/printf/printf.o
 .group         0x00000000        0x8 ./07_Soft_Component/printf/printf.o
 .group         0x00000000        0x8 ./07_Soft_Component/printf/printf.o
 .text          0x00000000        0x0 ./07_Soft_Component/printf/printf.o
 .data          0x00000000        0x0 ./07_Soft_Component/printf/printf.o
 .bss           0x00000000        0x0 ./07_Soft_Component/printf/printf.o
 .debug_macro   0x00000000      0x7f6 ./07_Soft_Component/printf/printf.o
 .debug_macro   0x00000000       0x16 ./07_Soft_Component/printf/printf.o
 .debug_macro   0x00000000       0x16 ./07_Soft_Component/printf/printf.o
 .debug_macro   0x00000000       0x44 ./07_Soft_Component/printf/printf.o
 .debug_macro   0x00000000      0x209 ./07_Soft_Component/printf/printf.o
 .debug_macro   0x00000000       0x3a ./07_Soft_Component/printf/printf.o
 .debug_macro   0x00000000       0x3a ./07_Soft_Component/printf/printf.o
 .debug_macro   0x00000000       0x26 ./07_Soft_Component/printf/printf.o
 .debug_macro   0x00000000      0x306 ./07_Soft_Component/printf/printf.o
 .debug_macro   0x00000000       0x10 ./07_Soft_Component/printf/printf.o
 .debug_macro   0x00000000     0x839f ./07_Soft_Component/printf/printf.o
 .debug_macro   0x00000000       0x4c ./07_Soft_Component/printf/printf.o
 .debug_macro   0x00000000       0x9a ./07_Soft_Component/printf/printf.o
 .group         0x00000000        0x8 ./07_Soft_Component/common/common.o
 .group         0x00000000        0x8 ./07_Soft_Component/common/common.o
 .group         0x00000000        0x8 ./07_Soft_Component/common/common.o
 .group         0x00000000        0x8 ./07_Soft_Component/common/common.o
 .group         0x00000000        0x8 ./07_Soft_Component/common/common.o
 .group         0x00000000        0x8 ./07_Soft_Component/common/common.o
 .group         0x00000000        0x8 ./07_Soft_Component/common/common.o
 .group         0x00000000        0x8 ./07_Soft_Component/common/common.o
 .group         0x00000000        0x8 ./07_Soft_Component/common/common.o
 .group         0x00000000        0x8 ./07_Soft_Component/common/common.o
 .group         0x00000000        0x8 ./07_Soft_Component/common/common.o
 .group         0x00000000        0x8 ./07_Soft_Component/common/common.o
 .text          0x00000000        0x0 ./07_Soft_Component/common/common.o
 .data          0x00000000        0x0 ./07_Soft_Component/common/common.o
 .bss           0x00000000        0x0 ./07_Soft_Component/common/common.o
 .text.NVIC_EnableIRQ
                0x00000000       0x2c ./07_Soft_Component/common/common.o
 .text.NVIC_DisableIRQ
                0x00000000       0x2c ./07_Soft_Component/common/common.o
 .text.NVIC_SetPriority
                0x00000000       0xe0 ./07_Soft_Component/common/common.o
 .bss.int_disable_level
                0x00000000        0x4 ./07_Soft_Component/common/common.o
 .text.init_critical
                0x00000000       0x14 ./07_Soft_Component/common/common.o
 .text.enter_critical
                0x00000000       0x20 ./07_Soft_Component/common/common.o
 .text.exit_critical
                0x00000000       0x28 ./07_Soft_Component/common/common.o
 .text.enable_irq
                0x00000000       0x30 ./07_Soft_Component/common/common.o
 .text.disable_irq
                0x00000000       0x30 ./07_Soft_Component/common/common.o
 .text.set_irq_priority
                0x00000000       0x60 ./07_Soft_Component/common/common.o
 .debug_macro   0x00000000      0x7f6 ./07_Soft_Component/common/common.o
 .debug_macro   0x00000000       0x16 ./07_Soft_Component/common/common.o
 .debug_macro   0x00000000       0x16 ./07_Soft_Component/common/common.o
 .debug_macro   0x00000000       0x44 ./07_Soft_Component/common/common.o
 .debug_macro   0x00000000      0x209 ./07_Soft_Component/common/common.o
 .debug_macro   0x00000000       0x3a ./07_Soft_Component/common/common.o
 .debug_macro   0x00000000       0x3a ./07_Soft_Component/common/common.o
 .debug_macro   0x00000000       0x26 ./07_Soft_Component/common/common.o
 .debug_macro   0x00000000      0x306 ./07_Soft_Component/common/common.o
 .debug_macro   0x00000000       0x10 ./07_Soft_Component/common/common.o
 .debug_macro   0x00000000     0x839f ./07_Soft_Component/common/common.o
 .debug_macro   0x00000000       0x4c ./07_Soft_Component/common/common.o
 .group         0x00000000        0x8 ./06_App_Component/light/light.o
 .group         0x00000000        0x8 ./06_App_Component/light/light.o
 .group         0x00000000        0x8 ./06_App_Component/light/light.o
 .group         0x00000000        0x8 ./06_App_Component/light/light.o
 .group         0x00000000        0x8 ./06_App_Component/light/light.o
 .group         0x00000000        0x8 ./06_App_Component/light/light.o
 .group         0x00000000        0x8 ./06_App_Component/light/light.o
 .group         0x00000000        0x8 ./06_App_Component/light/light.o
 .group         0x00000000        0x8 ./06_App_Component/light/light.o
 .group         0x00000000        0x8 ./06_App_Component/light/light.o
 .group         0x00000000        0x8 ./06_App_Component/light/light.o
 .group         0x00000000        0x8 ./06_App_Component/light/light.o
 .group         0x00000000        0x8 ./06_App_Component/light/light.o
 .group         0x00000000        0x8 ./06_App_Component/light/light.o
 .text          0x00000000        0x0 ./06_App_Component/light/light.o
 .data          0x00000000        0x0 ./06_App_Component/light/light.o
 .bss           0x00000000        0x0 ./06_App_Component/light/light.o
 .text.light_control
                0x00000000       0x28 ./06_App_Component/light/light.o
 .debug_macro   0x00000000      0x7f6 ./06_App_Component/light/light.o
 .debug_macro   0x00000000       0x16 ./06_App_Component/light/light.o
 .debug_macro   0x00000000       0x16 ./06_App_Component/light/light.o
 .debug_macro   0x00000000       0x44 ./06_App_Component/light/light.o
 .debug_macro   0x00000000      0x209 ./06_App_Component/light/light.o
 .debug_macro   0x00000000       0x3a ./06_App_Component/light/light.o
 .debug_macro   0x00000000       0x3a ./06_App_Component/light/light.o
 .debug_macro   0x00000000       0x26 ./06_App_Component/light/light.o
 .debug_macro   0x00000000      0x306 ./06_App_Component/light/light.o
 .debug_macro   0x00000000       0x10 ./06_App_Component/light/light.o
 .debug_macro   0x00000000     0x839f ./06_App_Component/light/light.o
 .debug_macro   0x00000000       0x4c ./06_App_Component/light/light.o
 .debug_macro   0x00000000       0x52 ./06_App_Component/light/light.o
 .group         0x00000000        0x8 ./05_Driver/uart/uart.o
 .group         0x00000000        0x8 ./05_Driver/uart/uart.o
 .group         0x00000000        0x8 ./05_Driver/uart/uart.o
 .group         0x00000000        0x8 ./05_Driver/uart/uart.o
 .group         0x00000000        0x8 ./05_Driver/uart/uart.o
 .group         0x00000000        0x8 ./05_Driver/uart/uart.o
 .group         0x00000000        0x8 ./05_Driver/uart/uart.o
 .group         0x00000000        0x8 ./05_Driver/uart/uart.o
 .group         0x00000000        0x8 ./05_Driver/uart/uart.o
 .group         0x00000000        0x8 ./05_Driver/uart/uart.o
 .group         0x00000000        0x8 ./05_Driver/uart/uart.o
 .group         0x00000000        0x8 ./05_Driver/uart/uart.o
 .group         0x00000000        0x8 ./05_Driver/uart/uart.o
 .text          0x00000000        0x0 ./05_Driver/uart/uart.o
 .data          0x00000000        0x0 ./05_Driver/uart/uart.o
 .bss           0x00000000        0x0 ./05_Driver/uart/uart.o
 .text.NVIC_DisableIRQ
                0x00000000       0x2c ./05_Driver/uart/uart.o
 .text.uart_sendN
                0x00000000       0x8c ./05_Driver/uart/uart.o
 .text.uart_send_string
                0x00000000       0x84 ./05_Driver/uart/uart.o
 .text.uart_reN
                0x00000000       0x9c ./05_Driver/uart/uart.o
 .text.uart_disable_re_int
                0x00000000       0x7c ./05_Driver/uart/uart.o
 .debug_macro   0x00000000      0x7f6 ./05_Driver/uart/uart.o
 .debug_macro   0x00000000       0x16 ./05_Driver/uart/uart.o
 .debug_macro   0x00000000       0x16 ./05_Driver/uart/uart.o
 .debug_macro   0x00000000       0x44 ./05_Driver/uart/uart.o
 .debug_macro   0x00000000      0x209 ./05_Driver/uart/uart.o
 .debug_macro   0x00000000       0x3a ./05_Driver/uart/uart.o
 .debug_macro   0x00000000       0x3a ./05_Driver/uart/uart.o
 .debug_macro   0x00000000       0x26 ./05_Driver/uart/uart.o
 .debug_macro   0x00000000      0x306 ./05_Driver/uart/uart.o
 .debug_macro   0x00000000       0x10 ./05_Driver/uart/uart.o
 .debug_macro   0x00000000     0x839f ./05_Driver/uart/uart.o
 .debug_macro   0x00000000       0x4c ./05_Driver/uart/uart.o
 .debug_macro   0x00000000       0x28 ./05_Driver/uart/uart.o
 .group         0x00000000        0x8 ./05_Driver/rtc/rtc.o
 .group         0x00000000        0x8 ./05_Driver/rtc/rtc.o
 .group         0x00000000        0x8 ./05_Driver/rtc/rtc.o
 .group         0x00000000        0x8 ./05_Driver/rtc/rtc.o
 .group         0x00000000        0x8 ./05_Driver/rtc/rtc.o
 .group         0x00000000        0x8 ./05_Driver/rtc/rtc.o
 .group         0x00000000        0x8 ./05_Driver/rtc/rtc.o
 .group         0x00000000        0x8 ./05_Driver/rtc/rtc.o
 .group         0x00000000        0x8 ./05_Driver/rtc/rtc.o
 .group         0x00000000        0x8 ./05_Driver/rtc/rtc.o
 .group         0x00000000        0x8 ./05_Driver/rtc/rtc.o
 .group         0x00000000        0x8 ./05_Driver/rtc/rtc.o
 .group         0x00000000        0x8 ./05_Driver/rtc/rtc.o
 .text          0x00000000        0x0 ./05_Driver/rtc/rtc.o
 .data          0x00000000        0x0 ./05_Driver/rtc/rtc.o
 .bss           0x00000000        0x0 ./05_Driver/rtc/rtc.o
 .text.NVIC_DisableIRQ
                0x00000000       0x2c ./05_Driver/rtc/rtc.o
 .text.rtc_reset_second_time
                0x00000000       0x18 ./05_Driver/rtc/rtc.o
 .text.rtc_disable_int
                0x00000000       0x14 ./05_Driver/rtc/rtc.o
 .debug_macro   0x00000000      0x7f6 ./05_Driver/rtc/rtc.o
 .debug_macro   0x00000000       0x16 ./05_Driver/rtc/rtc.o
 .debug_macro   0x00000000       0x16 ./05_Driver/rtc/rtc.o
 .debug_macro   0x00000000       0x44 ./05_Driver/rtc/rtc.o
 .debug_macro   0x00000000      0x209 ./05_Driver/rtc/rtc.o
 .debug_macro   0x00000000       0x3a ./05_Driver/rtc/rtc.o
 .debug_macro   0x00000000       0x3a ./05_Driver/rtc/rtc.o
 .debug_macro   0x00000000       0x26 ./05_Driver/rtc/rtc.o
 .debug_macro   0x00000000      0x306 ./05_Driver/rtc/rtc.o
 .debug_macro   0x00000000       0x10 ./05_Driver/rtc/rtc.o
 .debug_macro   0x00000000     0x839f ./05_Driver/rtc/rtc.o
 .debug_macro   0x00000000       0x4c ./05_Driver/rtc/rtc.o
 .group         0x00000000        0x8 ./05_Driver/gpio/gpio.o
 .group         0x00000000        0x8 ./05_Driver/gpio/gpio.o
 .group         0x00000000        0x8 ./05_Driver/gpio/gpio.o
 .group         0x00000000        0x8 ./05_Driver/gpio/gpio.o
 .group         0x00000000        0x8 ./05_Driver/gpio/gpio.o
 .group         0x00000000        0x8 ./05_Driver/gpio/gpio.o
 .group         0x00000000        0x8 ./05_Driver/gpio/gpio.o
 .group         0x00000000        0x8 ./05_Driver/gpio/gpio.o
 .group         0x00000000        0x8 ./05_Driver/gpio/gpio.o
 .group         0x00000000        0x8 ./05_Driver/gpio/gpio.o
 .group         0x00000000        0x8 ./05_Driver/gpio/gpio.o
 .group         0x00000000        0x8 ./05_Driver/gpio/gpio.o
 .group         0x00000000        0x8 ./05_Driver/gpio/gpio.o
 .text          0x00000000        0x0 ./05_Driver/gpio/gpio.o
 .data          0x00000000        0x0 ./05_Driver/gpio/gpio.o
 .bss           0x00000000        0x0 ./05_Driver/gpio/gpio.o
 .text.NVIC_EnableIRQ
                0x00000000       0x2c ./05_Driver/gpio/gpio.o
 .text.NVIC_DisableIRQ
                0x00000000       0x2c ./05_Driver/gpio/gpio.o
 .text.gpio_get
                0x00000000       0x54 ./05_Driver/gpio/gpio.o
 .text.gpio_pull
                0x00000000      0x11c ./05_Driver/gpio/gpio.o
 .text.gpio_enable_int
                0x00000000       0xb0 ./05_Driver/gpio/gpio.o
 .text.gpio_disable_int
                0x00000000       0x80 ./05_Driver/gpio/gpio.o
 .text.gpio_get_int
                0x00000000       0x58 ./05_Driver/gpio/gpio.o
 .text.gpio_clear_int
                0x00000000       0x60 ./05_Driver/gpio/gpio.o
 .text.gpio_clear_allint
                0x00000000       0x3c ./05_Driver/gpio/gpio.o
 .text.gpio_drive_strength
                0x00000000       0xb4 ./05_Driver/gpio/gpio.o
 .debug_macro   0x00000000      0x7f6 ./05_Driver/gpio/gpio.o
 .debug_macro   0x00000000       0x16 ./05_Driver/gpio/gpio.o
 .debug_macro   0x00000000       0x16 ./05_Driver/gpio/gpio.o
 .debug_macro   0x00000000       0x44 ./05_Driver/gpio/gpio.o
 .debug_macro   0x00000000      0x209 ./05_Driver/gpio/gpio.o
 .debug_macro   0x00000000       0x3a ./05_Driver/gpio/gpio.o
 .debug_macro   0x00000000       0x3a ./05_Driver/gpio/gpio.o
 .debug_macro   0x00000000       0x26 ./05_Driver/gpio/gpio.o
 .debug_macro   0x00000000      0x306 ./05_Driver/gpio/gpio.o
 .debug_macro   0x00000000       0x10 ./05_Driver/gpio/gpio.o
 .debug_macro   0x00000000     0x839f ./05_Driver/gpio/gpio.o
 .debug_macro   0x00000000       0x4c ./05_Driver/gpio/gpio.o
 .data          0x00000000        0x0 ./03_MCU/startup_MKL25Z4.o
 .bss           0x00000000        0x0 ./03_MCU/startup_MKL25Z4.o
 .group         0x00000000        0x8 ./03_MCU/system_MKL25Z4.o
 .group         0x00000000        0x8 ./03_MCU/system_MKL25Z4.o
 .group         0x00000000        0x8 ./03_MCU/system_MKL25Z4.o
 .group         0x00000000        0x8 ./03_MCU/system_MKL25Z4.o
 .group         0x00000000        0x8 ./03_MCU/system_MKL25Z4.o
 .group         0x00000000        0x8 ./03_MCU/system_MKL25Z4.o
 .group         0x00000000        0x8 ./03_MCU/system_MKL25Z4.o
 .group         0x00000000        0x8 ./03_MCU/system_MKL25Z4.o
 .group         0x00000000        0x8 ./03_MCU/system_MKL25Z4.o
 .group         0x00000000        0x8 ./03_MCU/system_MKL25Z4.o
 .text          0x00000000        0x0 ./03_MCU/system_MKL25Z4.o
 .data          0x00000000        0x0 ./03_MCU/system_MKL25Z4.o
 .bss           0x00000000        0x0 ./03_MCU/system_MKL25Z4.o
 .debug_macro   0x00000000      0x7f6 ./03_MCU/system_MKL25Z4.o
 .debug_macro   0x00000000       0x16 ./03_MCU/system_MKL25Z4.o
 .debug_macro   0x00000000       0x44 ./03_MCU/system_MKL25Z4.o
 .debug_macro   0x00000000      0x209 ./03_MCU/system_MKL25Z4.o
 .debug_macro   0x00000000       0x3a ./03_MCU/system_MKL25Z4.o
 .debug_macro   0x00000000       0x26 ./03_MCU/system_MKL25Z4.o
 .debug_macro   0x00000000      0x306 ./03_MCU/system_MKL25Z4.o
 .debug_macro   0x00000000       0x10 ./03_MCU/system_MKL25Z4.o
 .debug_macro   0x00000000     0x839f ./03_MCU/system_MKL25Z4.o
 .data          0x00000000        0x0 c:/freescale/kds_3.0.0/toolchain/bin/../lib/gcc/arm-none-eabi/4.8.4/armv6-m\libgcc.a(_udivsi3.o)
 .bss           0x00000000        0x0 c:/freescale/kds_3.0.0/toolchain/bin/../lib/gcc/arm-none-eabi/4.8.4/armv6-m\libgcc.a(_udivsi3.o)
 .data          0x00000000        0x0 c:/freescale/kds_3.0.0/toolchain/bin/../lib/gcc/arm-none-eabi/4.8.4/armv6-m\libgcc.a(_divsi3.o)
 .bss           0x00000000        0x0 c:/freescale/kds_3.0.0/toolchain/bin/../lib/gcc/arm-none-eabi/4.8.4/armv6-m\libgcc.a(_divsi3.o)
 .data          0x00000000        0x0 c:/freescale/kds_3.0.0/toolchain/bin/../lib/gcc/arm-none-eabi/4.8.4/armv6-m\libgcc.a(_dvmd_tls.o)
 .bss           0x00000000        0x0 c:/freescale/kds_3.0.0/toolchain/bin/../lib/gcc/arm-none-eabi/4.8.4/armv6-m\libgcc.a(_dvmd_tls.o)
 .data          0x00000000        0x0 c:/freescale/kds_3.0.0/toolchain/bin/../lib/gcc/arm-none-eabi/4.8.4/armv6-m\libgcc.a(_arm_cmpdf2.o)
 .bss           0x00000000        0x0 c:/freescale/kds_3.0.0/toolchain/bin/../lib/gcc/arm-none-eabi/4.8.4/armv6-m\libgcc.a(_arm_cmpdf2.o)
 .data          0x00000000        0x0 c:/freescale/kds_3.0.0/toolchain/bin/../lib/gcc/arm-none-eabi/4.8.4/armv6-m\libgcc.a(_aeabi_uldivmod.o)
 .bss           0x00000000        0x0 c:/freescale/kds_3.0.0/toolchain/bin/../lib/gcc/arm-none-eabi/4.8.4/armv6-m\libgcc.a(_aeabi_uldivmod.o)
 .data          0x00000000        0x0 c:/freescale/kds_3.0.0/toolchain/bin/../lib/gcc/arm-none-eabi/4.8.4/armv6-m\libgcc.a(_fixunsdfsi.o)
 .bss           0x00000000        0x0 c:/freescale/kds_3.0.0/toolchain/bin/../lib/gcc/arm-none-eabi/4.8.4/armv6-m\libgcc.a(_fixunsdfsi.o)
 .data          0x00000000        0x0 c:/freescale/kds_3.0.0/toolchain/bin/../lib/gcc/arm-none-eabi/4.8.4/armv6-m\libgcc.a(_fixunsdfdi.o)
 .bss           0x00000000        0x0 c:/freescale/kds_3.0.0/toolchain/bin/../lib/gcc/arm-none-eabi/4.8.4/armv6-m\libgcc.a(_fixunsdfdi.o)
 .data          0x00000000        0x0 c:/freescale/kds_3.0.0/toolchain/bin/../lib/gcc/arm-none-eabi/4.8.4/armv6-m\libgcc.a(bpabi.o)
 .bss           0x00000000        0x0 c:/freescale/kds_3.0.0/toolchain/bin/../lib/gcc/arm-none-eabi/4.8.4/armv6-m\libgcc.a(bpabi.o)
 .data          0x00000000        0x0 c:/freescale/kds_3.0.0/toolchain/bin/../lib/gcc/arm-none-eabi/4.8.4/armv6-m\libgcc.a(eqdf2.o)
 .bss           0x00000000        0x0 c:/freescale/kds_3.0.0/toolchain/bin/../lib/gcc/arm-none-eabi/4.8.4/armv6-m\libgcc.a(eqdf2.o)
 .data          0x00000000        0x0 c:/freescale/kds_3.0.0/toolchain/bin/../lib/gcc/arm-none-eabi/4.8.4/armv6-m\libgcc.a(gedf2.o)
 .bss           0x00000000        0x0 c:/freescale/kds_3.0.0/toolchain/bin/../lib/gcc/arm-none-eabi/4.8.4/armv6-m\libgcc.a(gedf2.o)
 .data          0x00000000        0x0 c:/freescale/kds_3.0.0/toolchain/bin/../lib/gcc/arm-none-eabi/4.8.4/armv6-m\libgcc.a(ledf2.o)
 .bss           0x00000000        0x0 c:/freescale/kds_3.0.0/toolchain/bin/../lib/gcc/arm-none-eabi/4.8.4/armv6-m\libgcc.a(ledf2.o)
 .data          0x00000000        0x0 c:/freescale/kds_3.0.0/toolchain/bin/../lib/gcc/arm-none-eabi/4.8.4/armv6-m\libgcc.a(muldf3.o)
 .bss           0x00000000        0x0 c:/freescale/kds_3.0.0/toolchain/bin/../lib/gcc/arm-none-eabi/4.8.4/armv6-m\libgcc.a(muldf3.o)
 .data          0x00000000        0x0 c:/freescale/kds_3.0.0/toolchain/bin/../lib/gcc/arm-none-eabi/4.8.4/armv6-m\libgcc.a(subdf3.o)
 .bss           0x00000000        0x0 c:/freescale/kds_3.0.0/toolchain/bin/../lib/gcc/arm-none-eabi/4.8.4/armv6-m\libgcc.a(subdf3.o)
 .data          0x00000000        0x0 c:/freescale/kds_3.0.0/toolchain/bin/../lib/gcc/arm-none-eabi/4.8.4/armv6-m\libgcc.a(fixdfsi.o)
 .bss           0x00000000        0x0 c:/freescale/kds_3.0.0/toolchain/bin/../lib/gcc/arm-none-eabi/4.8.4/armv6-m\libgcc.a(fixdfsi.o)
 .data          0x00000000        0x0 c:/freescale/kds_3.0.0/toolchain/bin/../lib/gcc/arm-none-eabi/4.8.4/armv6-m\libgcc.a(floatunsidf.o)
 .bss           0x00000000        0x0 c:/freescale/kds_3.0.0/toolchain/bin/../lib/gcc/arm-none-eabi/4.8.4/armv6-m\libgcc.a(floatunsidf.o)
 .data          0x00000000        0x0 c:/freescale/kds_3.0.0/toolchain/bin/../lib/gcc/arm-none-eabi/4.8.4/armv6-m\libgcc.a(_clzsi2.o)
 .bss           0x00000000        0x0 c:/freescale/kds_3.0.0/toolchain/bin/../lib/gcc/arm-none-eabi/4.8.4/armv6-m\libgcc.a(_clzsi2.o)
 .data          0x00000000        0x0 c:/freescale/kds_3.0.0/toolchain/bin/../lib/gcc/arm-none-eabi/4.8.4/armv6-m\libgcc.a(_muldi3.o)
 .bss           0x00000000        0x0 c:/freescale/kds_3.0.0/toolchain/bin/../lib/gcc/arm-none-eabi/4.8.4/armv6-m\libgcc.a(_muldi3.o)
 .data          0x00000000        0x0 c:/freescale/kds_3.0.0/toolchain/bin/../lib/gcc/arm-none-eabi/4.8.4/armv6-m\libgcc.a(_divdi3.o)
 .bss           0x00000000        0x0 c:/freescale/kds_3.0.0/toolchain/bin/../lib/gcc/arm-none-eabi/4.8.4/armv6-m\libgcc.a(_divdi3.o)
 .ARM.extab     0x00000000        0x0 c:/freescale/kds_3.0.0/toolchain/bin/../lib/gcc/arm-none-eabi/4.8.4/armv6-m\libgcc.a(_divdi3.o)
 .data          0x00000000        0x0 c:/freescale/kds_3.0.0/toolchain/bin/../lib/gcc/arm-none-eabi/4.8.4/armv6-m\libgcc.a(_udivdi3.o)
 .bss           0x00000000        0x0 c:/freescale/kds_3.0.0/toolchain/bin/../lib/gcc/arm-none-eabi/4.8.4/armv6-m\libgcc.a(_udivdi3.o)
 .ARM.extab     0x00000000        0x0 c:/freescale/kds_3.0.0/toolchain/bin/../lib/gcc/arm-none-eabi/4.8.4/armv6-m\libgcc.a(_udivdi3.o)
 .text          0x00000000        0x0 c:/freescale/kds_3.0.0/toolchain/bin/../lib/gcc/arm-none-eabi/4.8.4/../../../../arm-none-eabi/lib/armv6-m\libg.a(lib_a-memset.o)
 .data          0x00000000        0x0 c:/freescale/kds_3.0.0/toolchain/bin/../lib/gcc/arm-none-eabi/4.8.4/../../../../arm-none-eabi/lib/armv6-m\libg.a(lib_a-memset.o)
 .bss           0x00000000        0x0 c:/freescale/kds_3.0.0/toolchain/bin/../lib/gcc/arm-none-eabi/4.8.4/../../../../arm-none-eabi/lib/armv6-m\libg.a(lib_a-memset.o)
 .text          0x00000000        0x0 c:/freescale/kds_3.0.0/toolchain/bin/../lib/gcc/arm-none-eabi/4.8.4/../../../../arm-none-eabi/lib/armv6-m\libg.a(lib_a-strlen.o)
 .data          0x00000000        0x0 c:/freescale/kds_3.0.0/toolchain/bin/../lib/gcc/arm-none-eabi/4.8.4/../../../../arm-none-eabi/lib/armv6-m\libg.a(lib_a-strlen.o)
 .bss           0x00000000        0x0 c:/freescale/kds_3.0.0/toolchain/bin/../lib/gcc/arm-none-eabi/4.8.4/../../../../arm-none-eabi/lib/armv6-m\libg.a(lib_a-strlen.o)

Memory Configuration

Name             Origin             Length             Attributes
m_interrupts     0x00000000         0x00000100         xr
m_flash_config   0x00000400         0x00000010         xr
m_text           0x00000800         0x0001fbf0         xr
m_data           0x1ffff000         0x00004000         rw
*default*        0x00000000         0xffffffff

Linker script and memory map

LOAD ./08_Source/isr.o
LOAD ./08_Source/main.o
LOAD ./07_Soft_Component/printf/printf.o
LOAD ./07_Soft_Component/common/common.o
LOAD ./06_App_Component/light/light.o
LOAD ./05_Driver/uart/uart.o
LOAD ./05_Driver/rtc/rtc.o
LOAD ./05_Driver/gpio/gpio.o
LOAD ./03_MCU/startup_MKL25Z4.o
LOAD ./03_MCU/system_MKL25Z4.o
LOAD c:/freescale/kds_3.0.0/toolchain/bin/../lib/gcc/arm-none-eabi/4.8.4/armv6-m\libgcc.a
LOAD c:/freescale/kds_3.0.0/toolchain/bin/../lib/gcc/arm-none-eabi/4.8.4/../../../../arm-none-eabi/lib/armv6-m\libstdc++.a
LOAD c:/freescale/kds_3.0.0/toolchain/bin/../lib/gcc/arm-none-eabi/4.8.4/../../../../arm-none-eabi/lib/armv6-m\libm.a
START GROUP
LOAD c:/freescale/kds_3.0.0/toolchain/bin/../lib/gcc/arm-none-eabi/4.8.4/armv6-m\libgcc.a
LOAD c:/freescale/kds_3.0.0/toolchain/bin/../lib/gcc/arm-none-eabi/4.8.4/../../../../arm-none-eabi/lib/armv6-m\libg.a
LOAD c:/freescale/kds_3.0.0/toolchain/bin/../lib/gcc/arm-none-eabi/4.8.4/../../../../arm-none-eabi/lib/armv6-m\libc.a
END GROUP
                0x00000400                HEAP_SIZE = DEFINED (__heap_size__)?__heap_size__:0x400
                0x00000400                STACK_SIZE = DEFINED (__stack_size__)?__stack_size__:0x400

.interrupts     0x00000000       0xc0
                0x00000000                __VECTOR_TABLE = .
                0x00000000                . = ALIGN (0x4)
 *(.isr_vector)
 .isr_vector    0x00000000       0xc0 ./03_MCU/startup_MKL25Z4.o
                0x00000000                __isr_vector
                0x000000c0                . = ALIGN (0x4)

.flash_config   0x00000400       0x10
                0x00000400                . = ALIGN (0x4)
 *(.FlashConfig)
 .FlashConfig   0x00000400       0x10 ./03_MCU/startup_MKL25Z4.o
                0x00000410                . = ALIGN (0x4)

.text           0x00000800     0x3b2c
                0x00000800                . = ALIGN (0x4)
 *(.text)
 .text          0x00000800       0x4c ./03_MCU/startup_MKL25Z4.o
                0x00000800                Reset_Handler
                0x00000844                HardFault_Handler
                0x00000844                SysTick_Handler
                0x00000844                PendSV_Handler
                0x00000844                NMI_Handler
                0x00000844                I2C1_IRQHandler
                0x00000844                DMA2_IRQHandler
                0x00000844                TPM0_IRQHandler
                0x00000844                LLWU_IRQHandler
                0x00000844                TSI0_IRQHandler
                0x00000844                ADC0_IRQHandler
                0x00000844                Reserved39_IRQHandler
                0x00000844                SPI1_IRQHandler
                0x00000844                DefaultISR
                0x00000844                PORTD_IRQHandler
                0x00000844                TPM2_IRQHandler
                0x00000844                I2C0_IRQHandler
                0x00000844                MCG_IRQHandler
                0x00000844                Reserved20_IRQHandler
                0x00000844                USB0_IRQHandler
                0x00000844                PIT_IRQHandler
                0x00000844                SVC_Handler
                0x00000844                DMA3_IRQHandler
                0x00000844                DMA0_IRQHandler
                0x00000844                DAC0_IRQHandler
                0x00000844                Reserved45_IRQHandler
                0x00000844                TPM1_IRQHandler
                0x00000844                LVD_LVW_IRQHandler
                0x00000844                SPI0_IRQHandler
                0x00000844                PORTA_IRQHandler
                0x00000844                FTFA_IRQHandler
                0x00000844                LPTMR0_IRQHandler
                0x00000844                CMP0_IRQHandler
                0x00000844                DMA1_IRQHandler
 .text          0x0000084c       0x9c c:/freescale/kds_3.0.0/toolchain/bin/../lib/gcc/arm-none-eabi/4.8.4/armv6-m\libgcc.a(_udivsi3.o)
                0x0000084c                __aeabi_uidiv
                0x0000084c                __udivsi3
                0x000008d4                __aeabi_uidivmod
 .text          0x000008e8       0xc0 c:/freescale/kds_3.0.0/toolchain/bin/../lib/gcc/arm-none-eabi/4.8.4/armv6-m\libgcc.a(_divsi3.o)
                0x000008e8                __divsi3
                0x000008e8                __aeabi_idiv
                0x00000994                __aeabi_idivmod
 .text          0x000009a8        0x4 c:/freescale/kds_3.0.0/toolchain/bin/../lib/gcc/arm-none-eabi/4.8.4/armv6-m\libgcc.a(_dvmd_tls.o)
                0x000009a8                __aeabi_idiv0
                0x000009a8                __aeabi_ldiv0
 .text          0x000009ac       0x7c c:/freescale/kds_3.0.0/toolchain/bin/../lib/gcc/arm-none-eabi/4.8.4/armv6-m\libgcc.a(_arm_cmpdf2.o)
                0x000009ac                __aeabi_cdrcmple
                0x000009bc                __aeabi_cdcmple
                0x000009bc                __aeabi_cdcmpeq
                0x000009cc                __aeabi_dcmpeq
                0x000009d8                __aeabi_dcmplt
                0x000009ec                __aeabi_dcmple
                0x00000a00                __aeabi_dcmpgt
                0x00000a14                __aeabi_dcmpge
 .text          0x00000a28       0x40 c:/freescale/kds_3.0.0/toolchain/bin/../lib/gcc/arm-none-eabi/4.8.4/armv6-m\libgcc.a(_aeabi_uldivmod.o)
                0x00000a28                __aeabi_uldivmod
 .text          0x00000a68       0x40 c:/freescale/kds_3.0.0/toolchain/bin/../lib/gcc/arm-none-eabi/4.8.4/armv6-m\libgcc.a(_fixunsdfsi.o)
                0x00000a68                __aeabi_d2uiz
                0x00000a68                __fixunsdfsi
 .text          0x00000aa8       0x48 c:/freescale/kds_3.0.0/toolchain/bin/../lib/gcc/arm-none-eabi/4.8.4/armv6-m\libgcc.a(_fixunsdfdi.o)
                0x00000aa8                __fixunsdfdi
                0x00000aa8                __aeabi_d2ulz
 .text          0x00000af0       0x6c c:/freescale/kds_3.0.0/toolchain/bin/../lib/gcc/arm-none-eabi/4.8.4/armv6-m\libgcc.a(bpabi.o)
                0x00000af0                __gnu_ldivmod_helper
                0x00000b28                __gnu_uldivmod_helper
 .text          0x00000b5c       0x94 c:/freescale/kds_3.0.0/toolchain/bin/../lib/gcc/arm-none-eabi/4.8.4/armv6-m\libgcc.a(eqdf2.o)
                0x00000b5c                __nedf2
                0x00000b5c                __eqdf2
 .text          0x00000bf0       0xfc c:/freescale/kds_3.0.0/toolchain/bin/../lib/gcc/arm-none-eabi/4.8.4/armv6-m\libgcc.a(gedf2.o)
                0x00000bf0                __gedf2
                0x00000bf0                __gtdf2
 .text          0x00000cec       0xfc c:/freescale/kds_3.0.0/toolchain/bin/../lib/gcc/arm-none-eabi/4.8.4/armv6-m\libgcc.a(ledf2.o)
                0x00000cec                __ledf2
                0x00000cec                __ltdf2
 .text          0x00000de8      0x520 c:/freescale/kds_3.0.0/toolchain/bin/../lib/gcc/arm-none-eabi/4.8.4/armv6-m\libgcc.a(muldf3.o)
                0x00000de8                __aeabi_dmul
 .text          0x00001308      0x668 c:/freescale/kds_3.0.0/toolchain/bin/../lib/gcc/arm-none-eabi/4.8.4/armv6-m\libgcc.a(subdf3.o)
                0x00001308                __aeabi_dsub
 .text          0x00001970       0x68 c:/freescale/kds_3.0.0/toolchain/bin/../lib/gcc/arm-none-eabi/4.8.4/armv6-m\libgcc.a(fixdfsi.o)
                0x00001970                __aeabi_d2iz
 .text          0x000019d8       0x68 c:/freescale/kds_3.0.0/toolchain/bin/../lib/gcc/arm-none-eabi/4.8.4/armv6-m\libgcc.a(floatunsidf.o)
                0x000019d8                __aeabi_ui2d
 .text          0x00001a40       0x3c c:/freescale/kds_3.0.0/toolchain/bin/../lib/gcc/arm-none-eabi/4.8.4/armv6-m\libgcc.a(_clzsi2.o)
                0x00001a40                __clzsi2
 .text          0x00001a7c       0x44 c:/freescale/kds_3.0.0/toolchain/bin/../lib/gcc/arm-none-eabi/4.8.4/armv6-m\libgcc.a(_muldi3.o)
                0x00001a7c                __muldi3
                0x00001a7c                __aeabi_lmul
 .text          0x00001ac0      0x3b8 c:/freescale/kds_3.0.0/toolchain/bin/../lib/gcc/arm-none-eabi/4.8.4/armv6-m\libgcc.a(_divdi3.o)
                0x00001ac0                __divdi3
 .text          0x00001e78      0x384 c:/freescale/kds_3.0.0/toolchain/bin/../lib/gcc/arm-none-eabi/4.8.4/armv6-m\libgcc.a(_udivdi3.o)
                0x00001e78                __udivdi3
 *(.text*)
 .text.RTC_IRQHandler
                0x000021fc       0x9c ./08_Source/isr.o
                0x000021fc                RTC_IRQHandler
 .text.RTC_Seconds_IRQHandler
                0x00002298       0x14 ./08_Source/isr.o
                0x00002298                RTC_Seconds_IRQHandler
 .text.UART0_IRQHandler
                0x000022ac       0x40 ./08_Source/isr.o
                0x000022ac                UART0_IRQHandler
 .text.UART1_IRQHandler
                0x000022ec       0x40 ./08_Source/isr.o
                0x000022ec                UART1_IRQHandler
 .text.UART2_IRQHandler
                0x0000232c       0x40 ./08_Source/isr.o
                0x0000232c                UART2_IRQHandler
 .text.main     0x0000236c       0xbc ./08_Source/main.o
                0x0000236c                main
 .text.out_char
                0x00002428       0x20 ./07_Soft_Component/printf/printf.o
                0x00002428                out_char
 .text.printk_putc
                0x00002448       0x50 ./07_Soft_Component/printf/printf.o
 .text.printk_mkfloatstr
                0x00002498      0x398 ./07_Soft_Component/printf/printf.o
                0x00002498                printk_mkfloatstr
 .text.printk_mknumstr
                0x00002830      0x100 ./07_Soft_Component/printf/printf.o
 .text.printk_pad_zero
                0x00002930       0x38 ./07_Soft_Component/printf/printf.o
 .text.printk_pad_space
                0x00002968       0x38 ./07_Soft_Component/printf/printf.o
 .text.printk   0x000029a0      0xaa0 ./07_Soft_Component/printf/printf.o
                0x000029a0                printk
 .text.myprintf
                0x00003440       0x48 ./07_Soft_Component/printf/printf.o
                0x00003440                myprintf
 .text.SecAdd1  0x00003488       0x6c ./07_Soft_Component/common/common.o
                0x00003488                SecAdd1
 .text.light_init
                0x000034f4       0x2c ./06_App_Component/light/light.o
                0x000034f4                light_init
 .text.light_change
                0x00003520       0x1c ./06_App_Component/light/light.o
                0x00003520                light_change
 .text.NVIC_EnableIRQ
                0x0000353c       0x2c ./05_Driver/uart/uart.o
 .text.uart_init
                0x00003568      0x29c ./05_Driver/uart/uart.o
                0x00003568                uart_init
 .text.uart_send1
                0x00003804       0xa8 ./05_Driver/uart/uart.o
                0x00003804                uart_send1
 .text.uart_re1
                0x000038ac       0xc8 ./05_Driver/uart/uart.o
                0x000038ac                uart_re1
 .text.uart_enable_re_int
                0x00003974       0x7c ./05_Driver/uart/uart.o
                0x00003974                uart_enable_re_int
 .text.uart_get_re_int
                0x000039f0       0xe8 ./05_Driver/uart/uart.o
                0x000039f0                uart_get_re_int
 .text.uart_is_uartNo
                0x00003ad8       0x24 ./05_Driver/uart/uart.o
                0x00003ad8                uart_is_uartNo
 .text.NVIC_EnableIRQ
                0x00003afc       0x2c ./05_Driver/rtc/rtc.o
 .text.rtc_clockconfig
                0x00003b28       0x64 ./05_Driver/rtc/rtc.o
                0x00003b28                rtc_clockconfig
 .text.rtc_init
                0x00003b8c       0x98 ./05_Driver/rtc/rtc.o
                0x00003b8c                rtc_init
 .text.rtc_start
                0x00003c24       0x18 ./05_Driver/rtc/rtc.o
                0x00003c24                rtc_start
 .text.rtc_stop
                0x00003c3c       0x18 ./05_Driver/rtc/rtc.o
                0x00003c3c                rtc_stop
 .text.rtc_reset_alarm_time
                0x00003c54       0x18 ./05_Driver/rtc/rtc.o
                0x00003c54                rtc_reset_alarm_time
 .text.rtc_enable_int
                0x00003c6c       0x14 ./05_Driver/rtc/rtc.o
                0x00003c6c                rtc_enable_int
 .text.gpio_init
                0x00003c80       0xe8 ./05_Driver/gpio/gpio.o
                0x00003c80                gpio_init
 .text.gpio_set
                0x00003d68       0x80 ./05_Driver/gpio/gpio.o
                0x00003d68                gpio_set
 .text.gpio_reverse
                0x00003de8       0x54 ./05_Driver/gpio/gpio.o
                0x00003de8                gpio_reverse
 .text.gpio_get_port_pin
                0x00003e3c       0x34 ./05_Driver/gpio/gpio.o
                0x00003e3c                gpio_get_port_pin
 .text.SystemInit
                0x00003e70      0x1a0 ./03_MCU/system_MKL25Z4.o
                0x00003e70                SystemInit
 .text.memset   0x00004010       0x9c c:/freescale/kds_3.0.0/toolchain/bin/../lib/gcc/arm-none-eabi/4.8.4/../../../../arm-none-eabi/lib/armv6-m\libg.a(lib_a-memset.o)
                0x00004010                memset
 .text.strlen   0x000040ac       0x10 c:/freescale/kds_3.0.0/toolchain/bin/../lib/gcc/arm-none-eabi/4.8.4/../../../../arm-none-eabi/lib/armv6-m\libg.a(lib_a-strlen.o)
                0x000040ac                strlen
 *(.rodata)
 .rodata        0x000040bc       0xec ./08_Source/isr.o
 .rodata        0x000041a8       0x4c ./08_Source/main.o
 .rodata        0x000041f4       0x40 c:/freescale/kds_3.0.0/toolchain/bin/../lib/gcc/arm-none-eabi/4.8.4/armv6-m\libgcc.a(muldf3.o)
 *(.rodata*)
 .rodata.printk
                0x00004234       0xc8 ./07_Soft_Component/printf/printf.o
 .rodata.UART_ARR
                0x000042fc        0x8 ./05_Driver/uart/uart.o
 .rodata.PORT_ARR
                0x00004304       0x14 ./05_Driver/gpio/gpio.o
                0x00004304                PORT_ARR
 .rodata.GPIO_ARR
                0x00004318       0x14 ./05_Driver/gpio/gpio.o
                0x00004318                GPIO_ARR
 *(.glue_7)
 .glue_7        0x00000000        0x0 linker stubs
 *(.glue_7t)
 .glue_7t       0x00000000        0x0 linker stubs
 *(.eh_frame)
 *(.init)
 *(.fini)
                0x0000432c                . = ALIGN (0x4)

.vfp11_veneer   0x0000432c        0x0
 .vfp11_veneer  0x00000000        0x0 linker stubs

.v4_bx          0x0000432c        0x0
 .v4_bx         0x00000000        0x0 linker stubs

.iplt           0x0000432c        0x0
 .iplt          0x00000000        0x0 ./08_Source/isr.o

.ARM.extab
 *(.ARM.extab* .gnu.linkonce.armextab.*)

.ARM            0x0000432c        0x8
                0x0000432c                __exidx_start = .
 *(.ARM.exidx*)
 .ARM.exidx     0x0000432c        0x8 c:/freescale/kds_3.0.0/toolchain/bin/../lib/gcc/arm-none-eabi/4.8.4/armv6-m\libgcc.a(_divdi3.o)
 .ARM.exidx     0x00004334        0x0 c:/freescale/kds_3.0.0/toolchain/bin/../lib/gcc/arm-none-eabi/4.8.4/armv6-m\libgcc.a(_udivdi3.o)
                                  0x8 (size before relaxing)
                0x00004334                __exidx_end = .

.rel.dyn        0x00004334        0x0
 .rel.iplt      0x00000000        0x0 ./08_Source/isr.o

.ctors          0x00004334        0x0
                0x00004334                __CTOR_LIST__ = .
 *crtbegin.o(.ctors)
 *crtbegin?.o(.ctors)
 *(EXCLUDE_FILE(*crtend.o *crtend?.o) .ctors)
 *(SORT(.ctors.*))
 *(.ctors)
                0x00004334                __CTOR_END__ = .

.dtors          0x00004334        0x0
                0x00004334                __DTOR_LIST__ = .
 *crtbegin.o(.dtors)
 *crtbegin?.o(.dtors)
 *(EXCLUDE_FILE(*crtend.o *crtend?.o) .dtors)
 *(SORT(.dtors.*))
 *(.dtors)
                0x00004334                __DTOR_END__ = .

.preinit_array  0x00004334        0x0
                0x00004334                PROVIDE (__preinit_array_start, .)
 *(.preinit_array*)
                0x00004334                PROVIDE (__preinit_array_end, .)

.init_array     0x00004334        0x0
                0x00004334                PROVIDE (__init_array_start, .)
 *(SORT(.init_array.*))
 *(.init_array*)
                0x00004334                PROVIDE (__init_array_end, .)

.fini_array     0x00004334        0x0
                0x00004334                PROVIDE (__fini_array_start, .)
 *(SORT(.fini_array.*))
 *(.fini_array*)
                0x00004334                PROVIDE (__fini_array_end, .)
                0x00004334                __etext = .
                0x00004334                __DATA_ROM = .

.mtb            0x1ffff000        0x0
                0x1ffff000                . = ALIGN (0x8)
                0x1ffff000                _mtb_start = .
 *(.mtb_buf)
                0x1ffff000                . = ALIGN (0x8)
                0x1ffff000                _mtb_end = .

.data           0x1ffff000        0x8 load address 0x00004334
                0x1ffff000                . = ALIGN (0x4)
                0x1ffff000                __DATA_RAM = .
                0x1ffff000                __data_start__ = .
 *(.data)
 *(.data*)
 .data.table_irq_uart
                0x1ffff000        0x4 ./05_Driver/uart/uart.o
 .data.SystemCoreClock
                0x1ffff004        0x4 ./03_MCU/system_MKL25Z4.o
                0x1ffff004                SystemCoreClock
 *(.jcr*)
                0x1ffff008                . = ALIGN (0x4)
                0x1ffff008                __data_end__ = .
                0x0000433c                __DATA_END = (__DATA_ROM + (__data_end__ - __data_start__))

.igot.plt       0x1ffff008        0x0 load address 0x0000433c
 .igot.plt      0x00000000        0x0 ./08_Source/isr.o

.bss            0x1ffff008        0xc load address 0x0000433c
                0x1ffff008                . = ALIGN (0x4)
                0x1ffff008                __START_BSS = .
                0x1ffff008                __bss_start__ = .
 *(.bss)
 *(.bss*)
 *(COMMON)
 COMMON         0x1ffff008        0xb ./08_Source/isr.o
                0x1ffff008                AlarmTimes
                0x1ffff00c                SecondTimes
                0x1ffff010                g_time
                0x1ffff014                . = ALIGN (0x4)
 *fill*         0x1ffff013        0x1 
                0x1ffff014                __bss_end__ = .
                0x1ffff014                __END_BSS = .

.heap           0x1ffff014      0x404 load address 0x00004348
                0x1ffff018                . = ALIGN (0x8)
 *fill*         0x1ffff014        0x4 
                0x1ffff018                __end__ = .
                0x1ffff018                PROVIDE (end, .)
                0x1ffff018                __HeapBase = .
                0x1ffff418                . = (. + HEAP_SIZE)
 *fill*         0x1ffff018      0x400 
                0x1ffff418                __HeapLimit = .

.stack          0x1ffff418      0x400 load address 0x0000474c
                0x1ffff418                . = ALIGN (0x8)
                0x1ffff818                . = (. + STACK_SIZE)
 *fill*         0x1ffff418      0x400 
                0x20003000                __StackTop = (ORIGIN (m_data) + 0x4000)
                0x20002c00                __StackLimit = (__StackTop - STACK_SIZE)
                0x20003000                PROVIDE (__stack, __StackTop)

.ARM.attributes
                0x00000000       0x30
 *(.ARM.attributes)
 .ARM.attributes
                0x00000000       0x32 ./08_Source/isr.o
 .ARM.attributes
                0x00000032       0x32 ./08_Source/main.o
 .ARM.attributes
                0x00000064       0x32 ./07_Soft_Component/printf/printf.o
 .ARM.attributes
                0x00000096       0x32 ./07_Soft_Component/common/common.o
 .ARM.attributes
                0x000000c8       0x32 ./06_App_Component/light/light.o
 .ARM.attributes
                0x000000fa       0x32 ./05_Driver/uart/uart.o
 .ARM.attributes
                0x0000012c       0x32 ./05_Driver/rtc/rtc.o
 .ARM.attributes
                0x0000015e       0x32 ./05_Driver/gpio/gpio.o
 .ARM.attributes
                0x00000190       0x1b ./03_MCU/startup_MKL25Z4.o
 .ARM.attributes
                0x000001ab       0x32 ./03_MCU/system_MKL25Z4.o
 .ARM.attributes
                0x000001dd       0x1e c:/freescale/kds_3.0.0/toolchain/bin/../lib/gcc/arm-none-eabi/4.8.4/armv6-m\libgcc.a(_udivsi3.o)
 .ARM.attributes
                0x000001fb       0x1e c:/freescale/kds_3.0.0/toolchain/bin/../lib/gcc/arm-none-eabi/4.8.4/armv6-m\libgcc.a(_divsi3.o)
 .ARM.attributes
                0x00000219       0x1e c:/freescale/kds_3.0.0/toolchain/bin/../lib/gcc/arm-none-eabi/4.8.4/armv6-m\libgcc.a(_dvmd_tls.o)
 .ARM.attributes
                0x00000237       0x1e c:/freescale/kds_3.0.0/toolchain/bin/../lib/gcc/arm-none-eabi/4.8.4/armv6-m\libgcc.a(_arm_cmpdf2.o)
 .ARM.attributes
                0x00000255       0x1e c:/freescale/kds_3.0.0/toolchain/bin/../lib/gcc/arm-none-eabi/4.8.4/armv6-m\libgcc.a(_aeabi_uldivmod.o)
 .ARM.attributes
                0x00000273       0x2c c:/freescale/kds_3.0.0/toolchain/bin/../lib/gcc/arm-none-eabi/4.8.4/armv6-m\libgcc.a(_fixunsdfsi.o)
 .ARM.attributes
                0x0000029f       0x2c c:/freescale/kds_3.0.0/toolchain/bin/../lib/gcc/arm-none-eabi/4.8.4/armv6-m\libgcc.a(_fixunsdfdi.o)
 .ARM.attributes
                0x000002cb       0x2c c:/freescale/kds_3.0.0/toolchain/bin/../lib/gcc/arm-none-eabi/4.8.4/armv6-m\libgcc.a(bpabi.o)
 .ARM.attributes
                0x000002f7       0x2c c:/freescale/kds_3.0.0/toolchain/bin/../lib/gcc/arm-none-eabi/4.8.4/armv6-m\libgcc.a(eqdf2.o)
 .ARM.attributes
                0x00000323       0x2c c:/freescale/kds_3.0.0/toolchain/bin/../lib/gcc/arm-none-eabi/4.8.4/armv6-m\libgcc.a(gedf2.o)
 .ARM.attributes
                0x0000034f       0x2c c:/freescale/kds_3.0.0/toolchain/bin/../lib/gcc/arm-none-eabi/4.8.4/armv6-m\libgcc.a(ledf2.o)
 .ARM.attributes
                0x0000037b       0x2c c:/freescale/kds_3.0.0/toolchain/bin/../lib/gcc/arm-none-eabi/4.8.4/armv6-m\libgcc.a(muldf3.o)
 .ARM.attributes
                0x000003a7       0x2c c:/freescale/kds_3.0.0/toolchain/bin/../lib/gcc/arm-none-eabi/4.8.4/armv6-m\libgcc.a(subdf3.o)
 .ARM.attributes
                0x000003d3       0x2c c:/freescale/kds_3.0.0/toolchain/bin/../lib/gcc/arm-none-eabi/4.8.4/armv6-m\libgcc.a(fixdfsi.o)
 .ARM.attributes
                0x000003ff       0x2c c:/freescale/kds_3.0.0/toolchain/bin/../lib/gcc/arm-none-eabi/4.8.4/armv6-m\libgcc.a(floatunsidf.o)
 .ARM.attributes
                0x0000042b       0x1e c:/freescale/kds_3.0.0/toolchain/bin/../lib/gcc/arm-none-eabi/4.8.4/armv6-m\libgcc.a(_clzsi2.o)
 .ARM.attributes
                0x00000449       0x2c c:/freescale/kds_3.0.0/toolchain/bin/../lib/gcc/arm-none-eabi/4.8.4/armv6-m\libgcc.a(_muldi3.o)
 .ARM.attributes
                0x00000475       0x2c c:/freescale/kds_3.0.0/toolchain/bin/../lib/gcc/arm-none-eabi/4.8.4/armv6-m\libgcc.a(_divdi3.o)
 .ARM.attributes
                0x000004a1       0x2c c:/freescale/kds_3.0.0/toolchain/bin/../lib/gcc/arm-none-eabi/4.8.4/armv6-m\libgcc.a(_udivdi3.o)
 .ARM.attributes
                0x000004cd       0x2c c:/freescale/kds_3.0.0/toolchain/bin/../lib/gcc/arm-none-eabi/4.8.4/../../../../arm-none-eabi/lib/armv6-m\libg.a(lib_a-memset.o)
 .ARM.attributes
                0x000004f9       0x2c c:/freescale/kds_3.0.0/toolchain/bin/../lib/gcc/arm-none-eabi/4.8.4/../../../../arm-none-eabi/lib/armv6-m\libg.a(lib_a-strlen.o)
                0x00000001                ASSERT ((__StackLimit >= __HeapLimit), region m_data overflowed with stack and heap)
OUTPUT(KL25_RTC.elf elf32-littlearm)

.debug_info     0x00000000     0x2f6d
 .debug_info    0x00000000      0x283 ./08_Source/isr.o
 .debug_info    0x00000283      0x145 ./08_Source/main.o
 .debug_info    0x000003c8      0x67e ./07_Soft_Component/printf/printf.o
 .debug_info    0x00000a46      0x525 ./07_Soft_Component/common/common.o
 .debug_info    0x00000f6b      0x118 ./06_App_Component/light/light.o
 .debug_info    0x00001083      0xa79 ./05_Driver/uart/uart.o
 .debug_info    0x00001afc      0x7ba ./05_Driver/rtc/rtc.o
 .debug_info    0x000022b6      0x858 ./05_Driver/gpio/gpio.o
 .debug_info    0x00002b0e       0x97 ./03_MCU/startup_MKL25Z4.o
 .debug_info    0x00002ba5      0x3c8 ./03_MCU/system_MKL25Z4.o

.debug_abbrev   0x00000000      0xc2d
 .debug_abbrev  0x00000000       0xfb ./08_Source/isr.o
 .debug_abbrev  0x000000fb       0xa6 ./08_Source/main.o
 .debug_abbrev  0x000001a1      0x1f4 ./07_Soft_Component/printf/printf.o
 .debug_abbrev  0x00000395      0x193 ./07_Soft_Component/common/common.o
 .debug_abbrev  0x00000528       0x7b ./06_App_Component/light/light.o
 .debug_abbrev  0x000005a3      0x217 ./05_Driver/uart/uart.o
 .debug_abbrev  0x000007ba      0x176 ./05_Driver/rtc/rtc.o
 .debug_abbrev  0x00000930      0x1e9 ./05_Driver/gpio/gpio.o
 .debug_abbrev  0x00000b19       0x14 ./03_MCU/startup_MKL25Z4.o
 .debug_abbrev  0x00000b2d      0x100 ./03_MCU/system_MKL25Z4.o

.debug_aranges  0x00000000      0x2f8
 .debug_aranges
                0x00000000       0x40 ./08_Source/isr.o
 .debug_aranges
                0x00000040       0x20 ./08_Source/main.o
 .debug_aranges
                0x00000060       0x58 ./07_Soft_Component/printf/printf.o
 .debug_aranges
                0x000000b8       0x68 ./07_Soft_Component/common/common.o
 .debug_aranges
                0x00000120       0x30 ./06_App_Component/light/light.o
 .debug_aranges
                0x00000150       0x78 ./05_Driver/uart/uart.o
 .debug_aranges
                0x000001c8       0x68 ./05_Driver/rtc/rtc.o
 .debug_aranges
                0x00000230       0x88 ./05_Driver/gpio/gpio.o
 .debug_aranges
                0x000002b8       0x20 ./03_MCU/startup_MKL25Z4.o
 .debug_aranges
                0x000002d8       0x20 ./03_MCU/system_MKL25Z4.o

.debug_ranges   0x00000000      0x248
 .debug_ranges  0x00000000       0x30 ./08_Source/isr.o
 .debug_ranges  0x00000030       0x10 ./08_Source/main.o
 .debug_ranges  0x00000040       0x48 ./07_Soft_Component/printf/printf.o
 .debug_ranges  0x00000088       0x58 ./07_Soft_Component/common/common.o
 .debug_ranges  0x000000e0       0x20 ./06_App_Component/light/light.o
 .debug_ranges  0x00000100       0x68 ./05_Driver/uart/uart.o
 .debug_ranges  0x00000168       0x58 ./05_Driver/rtc/rtc.o
 .debug_ranges  0x000001c0       0x78 ./05_Driver/gpio/gpio.o
 .debug_ranges  0x00000238       0x10 ./03_MCU/system_MKL25Z4.o

.debug_macro    0x00000000     0x9ab7
 .debug_macro   0x00000000       0xdc ./08_Source/isr.o
 .debug_macro   0x000000dc      0x7f6 ./08_Source/isr.o
 .debug_macro   0x000008d2       0x16 ./08_Source/isr.o
 .debug_macro   0x000008e8       0x16 ./08_Source/isr.o
 .debug_macro   0x000008fe       0x44 ./08_Source/isr.o
 .debug_macro   0x00000942      0x209 ./08_Source/isr.o
 .debug_macro   0x00000b4b       0x3a ./08_Source/isr.o
 .debug_macro   0x00000b85       0x3a ./08_Source/isr.o
 .debug_macro   0x00000bbf       0x26 ./08_Source/isr.o
 .debug_macro   0x00000be5      0x306 ./08_Source/isr.o
 .debug_macro   0x00000eeb       0x10 ./08_Source/isr.o
 .debug_macro   0x00000efb     0x839f ./08_Source/isr.o
 .debug_macro   0x0000929a       0x4c ./08_Source/isr.o
 .debug_macro   0x000092e6       0x2e ./08_Source/isr.o
 .debug_macro   0x00009314       0x9a ./08_Source/isr.o
 .debug_macro   0x000093ae       0x52 ./08_Source/isr.o
 .debug_macro   0x00009400       0x28 ./08_Source/isr.o
 .debug_macro   0x00009428       0x22 ./08_Source/isr.o
 .debug_macro   0x0000944a       0x16 ./08_Source/isr.o
 .debug_macro   0x00009460       0xdc ./08_Source/main.o
 .debug_macro   0x0000953c       0xb8 ./07_Soft_Component/printf/printf.o
 .debug_macro   0x000095f4       0x28 ./07_Soft_Component/printf/printf.o
 .debug_macro   0x0000961c       0x9a ./07_Soft_Component/common/common.o
 .debug_macro   0x000096b6       0xb2 ./06_App_Component/light/light.o
 .debug_macro   0x00009768       0x22 ./06_App_Component/light/light.o
 .debug_macro   0x0000978a       0xa9 ./05_Driver/uart/uart.o
 .debug_macro   0x00009833       0xa9 ./05_Driver/rtc/rtc.o
 .debug_macro   0x000098dc       0x1c ./05_Driver/rtc/rtc.o
 .debug_macro   0x000098f8       0xa9 ./05_Driver/gpio/gpio.o
 .debug_macro   0x000099a1       0x4c ./05_Driver/gpio/gpio.o
 .debug_macro   0x000099ed       0x7e ./03_MCU/system_MKL25Z4.o
 .debug_macro   0x00009a6b       0x4c ./03_MCU/system_MKL25Z4.o

.debug_line     0x00000000     0x2751
 .debug_line    0x00000000      0x59d ./08_Source/isr.o
 .debug_line    0x0000059d      0x528 ./08_Source/main.o
 .debug_line    0x00000ac5      0x5eb ./07_Soft_Component/printf/printf.o
 .debug_line    0x000010b0      0x388 ./07_Soft_Component/common/common.o
 .debug_line    0x00001438      0x386 ./06_App_Component/light/light.o
 .debug_line    0x000017be      0x497 ./05_Driver/uart/uart.o
 .debug_line    0x00001c55      0x3ba ./05_Driver/rtc/rtc.o
 .debug_line    0x0000200f      0x442 ./05_Driver/gpio/gpio.o
 .debug_line    0x00002451       0x70 ./03_MCU/startup_MKL25Z4.o
 .debug_line    0x000024c1      0x290 ./03_MCU/system_MKL25Z4.o

.debug_str      0x00000000    0x3299d
 .debug_str     0x00000000    0x3207c ./08_Source/isr.o
                              0x3247e (size before relaxing)
 .debug_str     0x0003207c       0x2a ./08_Source/main.o
                              0x3242e (size before relaxing)
 .debug_str     0x000320a6      0x194 ./07_Soft_Component/printf/printf.o
                              0x322b4 (size before relaxing)
 .debug_str     0x0003223a      0x2dc ./07_Soft_Component/common/common.o
                              0x3216d (size before relaxing)
 .debug_str     0x00032516       0x4e ./06_App_Component/light/light.o
                              0x31f9f (size before relaxing)
 .debug_str     0x00032564      0x21f ./05_Driver/uart/uart.o
                              0x32301 (size before relaxing)
 .debug_str     0x00032783       0xa8 ./05_Driver/rtc/rtc.o
                              0x32360 (size before relaxing)
 .debug_str     0x0003282b      0x143 ./05_Driver/gpio/gpio.o
                              0x322bd (size before relaxing)
 .debug_str     0x0003296e       0x2f ./03_MCU/system_MKL25Z4.o
                              0x31dd1 (size before relaxing)

.comment        0x00000000       0x70
 .comment       0x00000000       0x70 ./08_Source/isr.o
                                 0x71 (size before relaxing)
 .comment       0x00000000       0x71 ./08_Source/main.o
 .comment       0x00000000       0x71 ./07_Soft_Component/printf/printf.o
 .comment       0x00000000       0x71 ./07_Soft_Component/common/common.o
 .comment       0x00000000       0x71 ./06_App_Component/light/light.o
 .comment       0x00000000       0x71 ./05_Driver/uart/uart.o
 .comment       0x00000000       0x71 ./05_Driver/rtc/rtc.o
 .comment       0x00000000       0x71 ./05_Driver/gpio/gpio.o
 .comment       0x00000000       0x71 ./03_MCU/system_MKL25Z4.o

.debug_frame    0x00000000      0xbd0
 .debug_frame   0x00000000       0xa8 ./08_Source/isr.o
 .debug_frame   0x000000a8       0x30 ./08_Source/main.o
 .debug_frame   0x000000d8      0x114 ./07_Soft_Component/printf/printf.o
 .debug_frame   0x000001ec      0x148 ./07_Soft_Component/common/common.o
 .debug_frame   0x00000334       0x70 ./06_App_Component/light/light.o
 .debug_frame   0x000003a4      0x190 ./05_Driver/uart/uart.o
 .debug_frame   0x00000534      0x140 ./05_Driver/rtc/rtc.o
 .debug_frame   0x00000674      0x1d0 ./05_Driver/gpio/gpio.o
 .debug_frame   0x00000844       0x30 ./03_MCU/system_MKL25Z4.o
 .debug_frame   0x00000874       0x20 c:/freescale/kds_3.0.0/toolchain/bin/../lib/gcc/arm-none-eabi/4.8.4/armv6-m\libgcc.a(_udivsi3.o)
 .debug_frame   0x00000894       0x20 c:/freescale/kds_3.0.0/toolchain/bin/../lib/gcc/arm-none-eabi/4.8.4/armv6-m\libgcc.a(_divsi3.o)
 .debug_frame   0x000008b4       0x2c c:/freescale/kds_3.0.0/toolchain/bin/../lib/gcc/arm-none-eabi/4.8.4/armv6-m\libgcc.a(_fixunsdfsi.o)
 .debug_frame   0x000008e0       0x2c c:/freescale/kds_3.0.0/toolchain/bin/../lib/gcc/arm-none-eabi/4.8.4/armv6-m\libgcc.a(_fixunsdfdi.o)
 .debug_frame   0x0000090c       0x50 c:/freescale/kds_3.0.0/toolchain/bin/../lib/gcc/arm-none-eabi/4.8.4/armv6-m\libgcc.a(bpabi.o)
 .debug_frame   0x0000095c       0x3c c:/freescale/kds_3.0.0/toolchain/bin/../lib/gcc/arm-none-eabi/4.8.4/armv6-m\libgcc.a(eqdf2.o)
 .debug_frame   0x00000998       0x38 c:/freescale/kds_3.0.0/toolchain/bin/../lib/gcc/arm-none-eabi/4.8.4/armv6-m\libgcc.a(gedf2.o)
 .debug_frame   0x000009d0       0x3c c:/freescale/kds_3.0.0/toolchain/bin/../lib/gcc/arm-none-eabi/4.8.4/armv6-m\libgcc.a(ledf2.o)
 .debug_frame   0x00000a0c       0x3c c:/freescale/kds_3.0.0/toolchain/bin/../lib/gcc/arm-none-eabi/4.8.4/armv6-m\libgcc.a(muldf3.o)
 .debug_frame   0x00000a48       0x3c c:/freescale/kds_3.0.0/toolchain/bin/../lib/gcc/arm-none-eabi/4.8.4/armv6-m\libgcc.a(subdf3.o)
 .debug_frame   0x00000a84       0x2c c:/freescale/kds_3.0.0/toolchain/bin/../lib/gcc/arm-none-eabi/4.8.4/armv6-m\libgcc.a(fixdfsi.o)
 .debug_frame   0x00000ab0       0x28 c:/freescale/kds_3.0.0/toolchain/bin/../lib/gcc/arm-none-eabi/4.8.4/armv6-m\libgcc.a(floatunsidf.o)
 .debug_frame   0x00000ad8       0x30 c:/freescale/kds_3.0.0/toolchain/bin/../lib/gcc/arm-none-eabi/4.8.4/armv6-m\libgcc.a(_muldi3.o)
 .debug_frame   0x00000b08       0x3c c:/freescale/kds_3.0.0/toolchain/bin/../lib/gcc/arm-none-eabi/4.8.4/armv6-m\libgcc.a(_divdi3.o)
 .debug_frame   0x00000b44       0x3c c:/freescale/kds_3.0.0/toolchain/bin/../lib/gcc/arm-none-eabi/4.8.4/armv6-m\libgcc.a(_udivdi3.o)
 .debug_frame   0x00000b80       0x30 c:/freescale/kds_3.0.0/toolchain/bin/../lib/gcc/arm-none-eabi/4.8.4/../../../../arm-none-eabi/lib/armv6-m\libg.a(lib_a-memset.o)
 .debug_frame   0x00000bb0       0x20 c:/freescale/kds_3.0.0/toolchain/bin/../lib/gcc/arm-none-eabi/4.8.4/../../../../arm-none-eabi/lib/armv6-m\libg.a(lib_a-strlen.o)
